:1000000000308A00B1290000831A0A28A500030ED7
:10001000A6000F288312A500030EA600A6140A0846
:10002000AD008A018313A50E0408A7002008A800CC
:100030002108A9002208AA002308AB002408AC006C
:1000400083128B1E25280B19B12827088400280845
:10005000A0002908A1002A08A2002B08A3002C0850
:10006000A4002D088A00260E83008312250EA618F0
:10007000831609000A108A100A1182070A342034F4
:10008000493472342034503475346C3473346534EC
:10009000203443346F3475346E34743465347234C0
:1000A0002034523453343234333432342D344334E4
:1000B000203456346534723431342E3430342034A4
:1000C0000A340D340A3400340A108A100A118207E7
:1000D0006334683431343A3400340A108A100A1117
:1000E0008207303475347334203400340A108A1097
:1000F0000A1182076334683432343A3400340A1007
:100100008A100A1182076334683433343A34003475
:100110000A108A100A1182076334683434343A347E
:1001200000340A108A100A1182073034753473348F
:1001300020340A340D3400347C08A1017B020318FA
:10014000A4287B08A000B028A0010830FD00FB0D0A
:10015000A00D7C0820020318A000A10DFD0BA7280C
:10016000D528B230810069086A02031CB9288516B7
:10017000BA28851269086B02031CC0280516C1281D
:10018000051269086C02031CC7288514C82885104D
:1001900069086D02031CCE280514CF280510E90A52
:1001A0006908FB000A30FC009C282008E9000B11BC
:1001B0008A1125287230840000080319EC280230C7
:1001C000A100A001A00BE228A10BE1289730A0001C
:1001D000A00BE828800BDF2800346E0884007A0822
:1001E0008000840A8001EE0A00340830F702031C04
:1001F0000429773084000310800C000803190429B7
:1002000002290000800B01290034F2013630720708
:1002100084008008031946293630720784000008DC
:10022000F3007308F400F40905150730F600753083
:10023000F700F520F60B1729F5017508073C031C9C
:100240003C297408A0007508A10003192B2903108C
:10025000A00CA10B272920080139A100211832295F
:100260000511332905150730F6007530F700F52024
:10027000F60B3529F50A1D2905110730F6007530F2
:10028000F700F520F60B3F29F20A0629003404088E
:10029000F900F31F54292D30FA00ED208403F209F0
:1002A000F309F20A0319F30A730EF038F500F507A3
:1002B000E23EF600323EF80073080F39F607F60703
:1002C000F807E93EF700F707F707720E0F39F7074F
:1002D000F807F70DF80DF809F80D72080F39F8074F
:1002E000F50D0730F4000A30F807F703031C7429F2
:1002F000F707F603031C7829F607F503031C7C298E
:10030000F507F403031C8029743084000730790555
:100310008407783004020319A9290008A000031DEE
:100320009729791AA729F919992920309A2908308B
:10033000F9003030A007F3010408F2002008F400AF
:100340002008FA00ED20720884007408A000840AD6
:1003500089290008A0003030A0072008FA00ED200D
:10036000003484011F3083051F1383161F149F144C
:100370001F159F15073083129F00703083168F0062
:100380008312EE01703083168F00073083129900BC
:100390008316050806308312A000A00BCD290000AB
:1003A00019088C111F1383161F109F101F119F1106
:1003B0000108C03907388100083065008312EF0159
:1003C0006F08273C031CEB2936306F078400203070
:1003D0008000EF0AE029EF016F08023C031CFC29B2
:1003E00033308500FA30F200DA200C308500FA3024
:1003F000F200DA20EF0AEC298B16C0308B044E3065
:1004000081003630EE002430F2002030FA00ED207A
:10041000F20B052A0A30FA00ED2005213630EE00F5
:100420000A30FA00ED200330F2002A30FA00ED2005
:10043000F20B152A0130F30073083A20F30AA000EA
:10044000FA00ED2022307302031D1C2A0330F40051
:100450002A30FA00ED20F40B282A0A30FA00ED20A9
:100460000D30FA00ED200A30FA00ED2005218B1640
:10047000F00170081D3C031C482A851D462A4230A5
:10048000A000A00B412A0000F00A472AF001392AF7
:100490008519482A8B12B101B00185195A2A0330F7
:1004A000A000A00B512A000000000130B007031883
:1004B000B10A4D2A851D672A0330A000A00B5E2AD1
:1004C000000000000130B0070318B10A5A2AB30136
:1004D000B2018519762A0330A000A00B6D2A000016
:1004E00000000130B2070318B30A692A851D832A68
:1004F0000330A000A00B7A2A000000000130B207F0
:100500000318B30A762AAF01AE018519922A033087
:10051000A000A00B892A000000000130AE070318DC
:10052000AF0A852A851D9F2A0330A000A00B962ABA
:10053000000000000130AE070318AF0A922AB5018F
:10054000B4018519AE2A0330A000A00BA52A000033
:1005500000000130B4070318B50AA12A851DBB2A83
:100560000330A000A00BB22A000000000130B40745
:100570000318B50AAE2A8B16B108031DC62A300827
:10058000773C031CC62A0330EA00E62AB108031DA3
:10059000D02A3008953C031CD02A0630EA00E62A0F
:1005A000B108031DDA2A30089F3C031CDA2A0A30FE
:1005B000EA00E62AB108031DE42A3008BD3C031C0A
:1005C000E42A0630EA00E62A0330EA00B308031DF5
:1005D000F02A3208773C031CF02A0330EB00102B82
:1005E000B308031DFA2A3208953C031CFA2A063088
:1005F000EB00102BB308031D042B32089F3C031C97
:10060000042B0A30EB00102BB308031D0E2B32080D
:10061000BD3C031C0E2B0630EB00102B0330EB000F
:10062000AF08031D1A2B2E08773C031C1A2B0A3027
:10063000EC003A2BAF08031D242B2E08953C031C1D
:10064000242B0330EC003A2BAF08031D2E2B2E0871
:100650009F3C031C2E2B0530EC003A2BAF08031DEA
:10066000382B2E08BD3C031C382B0730EC003A2BEE
:100670000730EC00B508031D442B3408773C031CFD
:10068000442B0330ED00642BB508031D4E2B3408BA
:10069000953C031C4E2B0630ED00642BB508031D62
:1006A000582B34089F3C031C582B0A30ED00642B58
:1006B000B508031D622B3408BD3C031C622B0630B9
:1006C000ED00642B0330ED003630EE00F2017208CD
:1006D0006420F20AA000FA00ED2004307202031D2B
:1006E000672B05213630EE00103084003108F3000E
:1006F0003008F200472105213630EE00F201720881
:100700006D20F20AA000FA00ED2004307202031DF1
:100710007F2B05213630EE00F20172087620F20AB6
:10072000A000FA00ED2004307202031D8D2B05217C
:100730003630EE00103084003308F3003208F20047
:10074000472105213630EE00F20172086D20F20AD1
:10075000A000FA00ED2004307202031DA52B052134
:100760003630EE00F20172087F20F20AA000FA0093
:10077000ED2004307202031DB32B05213630EE004C
:10078000103084002F08F3002E08F20047210521C5
:100790003630EE00F20172086D20F20AA000FA0075
:1007A000ED2004307202031DCB2B05213630EE0004
:1007B000F20172088820F20AA000FA00ED2004304D
:1007C0007202031DD92B05213630EE001030840053
:1007D0003508F3003408F200472105213630EE00D9
:1007E000F20172089120F20AA000FA00ED20063012
:0C07F0007202031DF12B0521372A630063
:02400E00C43CB0
:00000001FF
